:02000000F128E5
:10000800A00003088301B6000408B7000A08B80076
:100018008A015408BA005E08B9005F08BE00550896
:10002800BB005608C2005708C1005808C400590848
:10003800C3005A08C0005B08BD005C08BC005D082E
:10004800BF0083128B1CD028002393225408A900D8
:100058005508AA005608AB00A108031D3A2829082C
:10006800A2002A08A3002B08A400C128210BC1283C
:10007800E5229322D7012030D8004130D90016223A
:10008800D7018030D8003F30D9001622C030D700C1
:100098007F30D8004430D900DE215408AC00550820
:1000A800AD005608AE002C082D042E0403196E2846
:1000B8002C08D7002D08D8002E08D900D401A0306C
:1000C800D5004130D600DE215408A5005508A60009
:1000D80056087228A5017A30A6004430A7002208E5
:1000E800D7002308D8002408D9002908D4002A08F2
:1000F800D5002B08D6008E215408AF005508B00053
:100108005608B1002F08D4003008D5003108D600B1
:100118002D235408D7005508D8005608D9002508BB
:10012800D4002608D5002708D600BF210318B82810
:10013800D701D801D9012F08D4003008D5003108DB
:10014800D600BF210318B2282508D7002608D800F2
:100158002708D900223084006B21C1282508D70040
:100168002608D8002708BD282F08D7003008D8004F
:100178003108D900223084006D2183122208D4006E
:100188002308D5002408D60057225408B200550881
:10019800B300A2228B1083123A08D4003908DE007B
:1001A8003E08DF003B08D5004208D6004108D700CA
:1001B8004408D8004308D9004008DA003D08DB00AD
:1001C8003C08DC003F08DD003708840038088A0056
:1001D80036088300A00E200E090021308400363036
:1001E800FD208316FF2390008301C62A04068001A0
:1001F800840A0406031DFA28640000340310FF3043
:10020800D407D409031CD507D509031CD607D6097A
:10021800031CD707D7090800D501D601D701D41F79
:100228007F2AD503D603D7037A2AD501D601D70169
:100238007F2ADC01550D560DDA005A0803192829C2
:10024800DC0DD601D5170800D401D501D60100343C
:10025800DC10580D590DDB005B0803193829031809
:10026800DC14D901D8170800DB01D701D801D9015E
:1002780008005A0803192829D513DC0C5A0CD60093
:100288000318D517962ADA08031D5B29D401D5016E
:10029800D601962A56030319D40A0319D50A031955
:1002A800D60A0310D60CD50CD40CDA0A4729D6087E
:1002B800031D4E295408550403194A29D51B3D2905
:1002C800DA0303194A290310D40DD50D62298030A9
:1002D800D9060008D400840A0008D500840A00085A
:1002E800D60091295A085B02031C852903190800C6
:1002F8000310D60CD50CD40CDA0A5A085B027A29FA
:100308000310D90CD80CD70CDB0A5A085B06031962
:10031800080084298030D90684011D212C217621EA
:100328005C1C9E29D409D509D609D40A0319D50A13
:100338000319D60ADC1CA829D709D809D909D70A6C
:100348000319D80A0319D90A5708D40758080318F3
:10035800580FD50759080318590FD607DC01D61FBF
:100368004729D409D509D609D40A0319D50A031986
:10037800D60A5C1447295608590680390319C82932
:10038800590D590801380800D61359087F39560203
:10039800031DD62958085502031DD62957085402AB
:1003A8000319080003080238D91B013A830003180F
:1003B8008038080084011D212C21DD01DE01DF01C8
:1003C800DA08031908005B08031908005A02773E87
:1003D800DA005C0CDC061830D9000310DD0DDE0DE8
:1003E800DF0D5608031D002A58085502031DFE2973
:1003F80057085402031C0A2A5708D4025808031C39
:10040800580FD502031CD6035D140310D40DD50D67
:10041800D60DD90BF1295D08D4005E08D5005F0818
:10042800D600472984011D212C21DD01DE01DF01D1
:100438000730D9000310D80CD70C031C2E2A5408F7
:10044800DD0755080318550FDE0756080318560F21
:10045800DF070310D40DD50DD60DD90B1E2A093090
:10046800D9003A2A0310DF0CDE0CDD0C0310D80C7F
:10047800D70C031C492A5408DD0755080318550FE3
:10048800DE0756080318560FDF07D90B362A5C0C0F
:10049800DC065D08D4005E08D5005F08D6007A3017
:1004A8005B07DA07472984011D21D7018230DA0763
:1004B800DA1B2829F030DA07DA1B732A18305A02B7
:1004C80003182829DA08031D6C2A5C180221080081
:1004D800DA030310D40DD50DD60DD70D662A0310F7
:1004E800D60CD50CD40CDA0F732A692AD71F7F2AA9
:1004F8005C140221802ADC018E30DA008401D708DE
:10050800031947290310D70CD60CD50CD40CDA0ADA
:10051800832AD601D51BD6035608D7007A2AD601D6
:10052800D7017F2A84080319003456088000840301
:100538005508800084035408800000340230831278
:100548003302BC3003193202031C0800083033029E
:10055800FD3003193202031808003308D5003208A9
:10056800D400D409D5095408B4005508B5008F0043
:1005780034088E000C10101485140C1CC12A851028
:10058800101008008312A80183121923A1018316F1
:1005980001170B160B118B108B17D62A0B1DD62A99
:1005A800A80A0B1183122808D4001921D701C030DA
:1005B800D8003F30D900BF21031CD22AA101A10ACB
:1005C800E42A8C3083129F00183083169F00831210
:1005D8001F142130B400B40BEF2A9F149F18F22A7D
:1005E8001E08B30083161E088312B2001F103308BA
:1005F800D5003208D400080083128F018E01101430
:100608000519042B10100F088312B300B2010E084D
:10061800D400D5013208D4070318D50A3308D50702
:100628002730D4070318D50A08008316FF23900043
:1006380083123D308316850018309F00FF308312E7
:100648009900043090004730831681009514831276
:060658000800D613003477
:084000000000080001000000AF
:02400E00843FED
:00000001FF
